:020000040000FA
:02000000642872
:08000800F000030E8312F10069
:100010005D218B180D280B181A28061C5528221450
:10002000A5012613A2108511861F0530861B2030DE
:10003000A6005E282308060603195528A300231AE4
:100040002828A31A2E28231B3428A31B3E28552812
:10005000061E5528221855284B304F28861E552835
:100060002218552851304F28061B5528221C552888
:100070002210861F0B30861B83304F28861B412899
:100080004A28A5012613A2108511221C83302218AC
:1000900007304F28221C0830221805304F28A700AF
:1000A000260840392704A6005E280608A3008B1006
:1000B0000B10710E8300F00E700E09000608A300ED
:1000C0008B100B108B178A281F149F101F159F125F
:1000D0008316F6308500831285018316FE30920068
:1000E0008312003095009701971517158316861116
:1000F00083121210921012150608A300A601A20185
:100100008316011783120B168B158B100B108B1790
:1001100059215921A608031D93289508031D9328EA
:10012000630000000000261F98289F1B9828851553
:10013000261CB028A61E9E284321A612A61CA8286D
:10014000261DCF202619D6202610A6102611B0284D
:10015000261DDD202619E4202610A6102611B02821
:10016000261EB7282612051EB7282215EB20261FAB
:10017000BD280B2185112613A214A61DC1282421F8
:10018000A611A61EC5284321A612A61FCA28A6137B
:100190004A21DD2005145D2105105D218A28FF30EC
:1001A000150203190800950A6D21CF28FF301502AA
:1001B00003190800950A7121D62800301502031989
:1001C000080095036D21DD28003015020319080091
:1001D00095037121E428592159215921F220F22057
:1001E000F22008009501FF30950005146521652176
:1001F000950105105D2104309507692188301502AD
:10020000031DFB2805145D21043095026921031D9F
:10021000042905100800250803191029C100162912
:100220000F30C100003022190430C1022211051024
:100230004108A500592159215921592105145D2151
:100240000510A50B1A290800950803190800FF30AE
:10025000150203192E29950A6D2127291E30C00089
:100260000030A2180F30C002A21005104008A400F0
:10027000592159215921592105145D210510A40B3B
:100280003829DD20080046301502031908009503BF
:10029000712143290F30A9003C30B00059210514C9
:1002A0005921592159210510B00B4E29A90B4C2970
:1002B0000800FA30A000752108003230A000752136
:1002C00008002830A000752108001E30A00075210C
:1002D00008000F30A000752108000A30A000752129
:1002E00008000530A00075210800F930A1000000C9
:1002F00000000000000000000000000000000000FE
:1003000000000000000000000000000000000000ED
:0A031000A10B7729A00B7529080046
:02400E00023F6F
:00000001FF
